:020000040000FA
:02000000412895
:08000800FE000308FF00D40B09
:100010000B2853150F280B118B16273081007F08F2
:100020008300FE0E7E0E0900820700340034003487
:10003000003400341B3477344034003435346734B2
:10004000E03400346A34CF34C03400349A341D3480
:1000500020340034D5349F34803401341334B23426
:100060002034013440346F34403401347B34CA349A
:1000700090340134AB343F3400340134C934C334D8
:10008000803407309F00EB2383168113FF308500F7
:1000900086018312A901AA01AB01AC01AD010F23B6
:1000A0000F23E92009215314CA01051A5B28CA1439
:1000B0004222CA105310522183169B01D3231A08DF
:1000C000F400D3231A08F500D3231A08F600D3232B
:1000D0001A08F700D3231A08F000D3231A08F100F6
:1000E000D3231A08F200D3231A08F300831229231A
:1000F0005723D8220F230508C30003304305C2004D
:10010000D301C401C8015318C529831607308100E3
:10011000831204308B008B178B162730810012302E
:10012000D400C521D3189D287030CB007130CC008D
:100130007230CD007330CE00D314B101B001AF01E5
:100140004A19A928CA19AE284A1AB5280130AE00A2
:10015000BB28E830AE000330AF00BB28A030AE00B3
:100160008630AF000130B000BB280F30B000423005
:10017000AF004030AE00C418BF28B221C12875219D
:100180008D2129235723D8220F238328EB23051AF7
:1001900008000430C807D73048070318C801D72023
:1001A00029235723D8220F23051ED42808004808E6
:1001B0001420F300C80A48081420F200C80A4808AE
:1001C0001420F100C80A48081420F0000330C802C7
:1001D0000800E223033086000616E22306120330ED
:1001E00086000616E5230612033086000616E52370
:1001F0000612023086000616E82306122830A423D1
:100200000830A4230130A4230630A4230C30A423F7
:1002100008008030A4235030A8234930A82343305D
:10022000A8234530A8234C30A8236730A823653085
:10023000A8236E30A8238830BB00A4233730A8231E
:100240002E30A8233430A8232D30A8233630A823FD
:100250003030A8232030A8232030A823C030A42386
:100260002030A8232030A8232030A8232030A82322
:100270002030A8232030A8232030A8232030A82312
:100280002030A8232030A8232030A8232030A82302
:100290002030A8232030A8232030A8232030A823F2
:1002A000D7230800C030A4235330A8235430A823F8
:1002B0004530A8235030A8233A30A8233130A82352
:1002C0004830A8237A30A8232030A8232030A82340
:1002D0002030A8232030A8232030A8232030A823B2
:1002E0002030A8232030A82308002E08F007031C84
:1002F0007E29F10F7E29F20F7E29F30A2F08F107DC
:10030000031C8529F20F8529F30A3008F207031C24
:100310008A29F30A3108F3070800FC307307031831
:10032000A92903307302031CB1296C30720703182A
:10033000A92993307202031CB12978307107031880
:10034000A92987307102031CB12900307002031CF7
:10035000B1290030F0008730F1009330F200033013
:10036000F3000800AE09AF09B009B109AE0FBD290D
:10037000AF0FBD29B00FBD29B10A7521F31FC429E4
:10038000F001F101F201F30108005318C9295319D2
:10039000AA22CA1CF7210508C300ED23050843065D
:1003A000031DC92903304305C10042060319C529AD
:1003B0000310C20D4108C20642080239C5004406B6
:1003C000C401C218EB294108C200C7034718C52958
:1003D000C718C529F4290230C4004108C200C70A61
:1003E0004718C529C718C5294108C2000800851942
:1003F0003F2AEB2385193F2A4A1EFF292F2ACA1DAF
:10040000102A4A16CA11C630A4234D30A8234830FA
:10041000A8237A30A8232030A8232030A8233C2A00
:100420004A1D212ACA154A11C630A4233030A823F8
:100430003030A8236B30A8234830A8237A30A82373
:100440003C2A4A15C630A4236B30A8234830A82381
:100450007A30A8232030A8232030A8233C2A4A122F
:10046000C630A4234830A8237A30A8232030A823FC
:100470002030A8232030A823851D3C2A0800051E13
:10048000C62008008030F0009630F1009830F2006D
:100490000030F30083169B01D3231A08F400D32302
:1004A0001A08F500D3231A08F600D3231A08F70018
:1004B000831229235723C430BB00A4234330BB003D
:1004C000A8234130BB00A8234C30BB00A823D8226E
:1004D0000F23C521B101B001AF011030AE004319A7
:1004E000732A8030AE000000C418812AAE09AF091B
:1004F000B009B109AE0F812AAF0F812AB00F812A4E
:10050000B10A2E08F407031C8A2AF50F8A2AF60F6F
:100510008A2AF70A2F08F507031C912AF60F912A59
:10052000F70A3008F607031C962AF70A3108F7077E
:10053000051E672A740883169B019A00C623750856
:100540009A00C62376089A00C62377089A00C62325
:10055000831208008B13D3105311CB30A423203007
:10056000A8232030A8232030A8232030A8232A3015
:10057000A823DC23DC23CB30A4232030A823203085
:10058000A8232030A8232030A8232030A8238316B6
:1005900004309B0070089A00C62371089A00C62395
:1005A00072089A00C62373089A00C62383120800B3
:1005B000A901AA01AB01AC01AD012030B40074085F
:1005C000B7007508B8007608B9007708BA000310BC
:1005D000371C012B7008AA07031CF32AAB0FF32A60
:1005E000AC0FF32AAD0A7108AB07031CFA2AAC0F53
:1005F000FA2AAD0A7208AC07031CFF2AAD0A730879
:10060000AD07AD0CAC0CAB0CAA0CA90CBA0CB90C18
:10061000B80CB70CB40BE72A0130AD000800293044
:1006200084000008B6000830B500B60C031C1C2B73
:100630008615061506111F2B861106150611B50B1A
:10064000152B840A2E300402031C112B86178613E7
:1006500008002030B200A401A501A601A701A8014D
:100660000310F00DF10DF20DF30D03187014A40D2D
:10067000A50DA60DA70DA80DB203031D402B080064
:10068000243084004C23840A4C23840A4C23840A9B
:100690004C23840A4C23302B03300007B300B319DA
:1006A000800030300007B300B31B800008008030AA
:1006B000A4232030A823270E0F39303EA823270873
:1006C0000F39303EA8232C30A823260E0F39303E98
:1006D000A82326080F39303EA823250E0F39303EB7
:1006E000A8232E30A8238830A42325080F39303EB4
:1006F000A823240E0F39303EA82324080F39303E9A
:10070000A8232030A8236B30A8234830A8237A30B0
:10071000A8232030A823080086018316083086000D
:10072000831206138616FF30BD0006160608BC00AD
:10073000061200000000061600000612BD03031991
:10074000A32BBC19952B0800BB00C9010613AB2BCA
:10075000BB00491406178C238601831600308600DF
:1007600083128612061349180617F03086053B0ED1
:100770000F398604061600000612F03086053B0885
:100780000F39860406160000061208001C158B138C
:1007900055309D00AA309D009C149C18CD2B9C17B1
:1007A0001C119B0A08001C141A089B0A0800DC2371
:1007B000DC23DC23DC230800DF23DF230800FF30F9
:1007C000BD00EF2B8030BD00EF2B4030BD00EF2B84
:1007D0002030BD00EF2B1030BD000230BD00FF30D7
:0C07E000BE00BE0BF12BBD0BEF2B080080
:02400E00303F41
:10420000DE006500DC00170028000100D600000079
:10421000000000000000000000000000000000009E
:10422000000000000000000000000000000000008E
:10423000000000000000000000000000000000007E
:10424000000000000000000000000000000000006E
:10425000000000000000000000000000000000005E
:10426000000000000000000000000000000000004E
:10427000000000000000000000000000000000003E
:10428000000000000000000000000000000000002E
:10429000000000000000000000000000000000001E
:1042A000000000000000000000000000000000000E
:1042B00000000000000000000000000000000000FE
:1042C00000000000000000000000000000000000EE
:1042D00000000000000000000000000000000000DE
:1042E00000000000000000000000000000000000CE
:00000001FF
